:040000008A11112828
:10000800FE00030EF3000408F4000A08F50083124A
:1000180003137F08F6008A1123288A111328FB018D
:10002800F701F801F901FA01A001A101A201A30158
:10003800A401A501A601A70183018A11AC288B1A86
:100048000B1DA1287A08F1007908F000F90A0319B4
:10005800FA0A00307102653003197002031C9E28E9
:10006800F901FA012308031D46282208031D462822
:1000780003302102031D4428E9302002031D4428CF
:10008800031C5A280030A3000030A2000030A10051
:100098000030A0000310871D0314031C5728831287
:1000A800031387155A288312031387112708031D82
:1000B8006A282608031D6A2803302502031D6828BC
:1000C800E9302402031D6828031C83280130F70047
:1000D8000030F8000030A7000030A6000030A5006E
:1000E8000030A4000310071E0314031C7F2883128A
:1000F800031307169E288312031307129E28051A56
:100108009E287708780403199E288716851A9E2842
:100118000714F701F8010330F2000830F1007830D5
:10012800F000F00B9528F10B9528F20B9528831217
:1001380003130710B23081000B117608FF00750811
:100148008A0074088400730E8300FE0E7E0E090078
:10015800831603130F168F160F1707308312031316
:1001680099008316031391013F30850087010730FA
:100178008100B2308312031381008B160B118B1789
:1001880087120712871107118710051DCE288714BB
:100198000711D02887100715050C0139A800003071
:1001A8007B18013028060319EA280130A00700301F
:1001B80003180130A107003003180130A2070030EE
:1001C80003180130A3077B1085187B1483120313CF
:1001D80005080139A8000030FB180130280603196A
:1001E80006290130A407003003180130A5070030A4
:1001F80003180130A607003003180130A707FB10C9
:100208000518FB1483120313051EC9280310851D46
:100218000314031C1329831203138716C928831296
:0602280003138712C92830
:02400E0004FFAD
:00000001FF
